:020000020000FC
:100000000AC018951895189518951895189518956B
:100010001895189518950FED0DBF0CEF07BB00E272
:1000200001BB01E00FD005E00DD004E00BD006E0ED
:1000300009D002E007D00AE005D008E003D009E0CB
:1000400001D0EFCFC798C598C398C29800FDC79A52
:1000500001FDC59A02FDC39A03FDC29A04D095988A
:100060004599959A08950F931F9300E018EC0000AE
:1000700000001A95E1F70A95C9F71F910F910895AD
:00000001FF
